:020000040000FA
:02000000A32E2D
:08000800803120002330950037
:10001000A10A103021020318A1012014A20F1328F5
:10002000A30F1328A0143D08003E03192D282E1CF1
:100030002B288E018E14232301302D2300001E3027
:10004000A4008E1007302D238E1406302D23A40B10
:1000500021288E10742823232F28182314230A30D4
:10006000A500BA21C021CE211C2321080319782024
:100070000130210203198720023021020319962042
:10008000033021020319A520043021020319B420F2
:10009000053021020319C320063021020319D220A2
:1000A000073021020319E120083021020319F02052
:1000B000093021020319FF200A30210203190E2101
:1000C0000B30210203191D210C30210203192C21B0
:1000D0000D30210203193B210E30210203194A2160
:1000E0000F302102031959218C018D010B110900D8
:1000F00000308E00F03084002030850091213030B7
:100100008400213085006821A50B7A280800013081
:100110008E0070308400213085009121B030840041
:10012000213085006821A50B8928080020308E0029
:10013000F83084002030850091213830840021304F
:1001400085006821A50B9828080021308E007830A2
:100150008400213085009121B83084002130850051
:100160006821A50BA728080040308E0000308400CD
:1001700021308500912140308400213085006821A4
:10018000A50BB628080041308E0080308400213055
:1001900085009121C0308400213085006821A50BA5
:1001A000C528080060308E000830840021308500AA
:1001B000912148308400213085006821A50BD42886
:1001C000080061308E008830840021308500912144
:1001D000C8308400213085006821A50BE328080081
:1001E00080308E0010308400213085009121503005
:1001F0008400213085006821A50BF2280800813099
:100200008E0090308400213085009121D030840010
:10021000213085006821A50B01290800A0308E003F
:10022000183084002130850091215830840021301D
:1002300085006821A50B10290800A1308E00983098
:100240008400213085009121D83084002130850040
:100250006821A50B1F290800C0308E0020308400C3
:100260002130850091216030840021308500682193
:10027000A50B2E290800C1308E00A030840021304B
:1002800085009121E0308400213085006821A50B94
:100290003D290800E0308E002830840021308500A0
:1002A000912168308400213085006821A50B4C29FC
:1002B0000800E1308E00A8308400213085009121B3
:1002C000E8308400213085006821A50B5B290800F7
:1002D0008C011508000203180C1412001508000206
:1002E00003188C1412001508000203180C151200D4
:1002F0001508000203188C151200150800020318D7
:100300000C1612001508000203188C1612001508AE
:10031000000203180C1712001508000203188C17AE
:1003200008008D011508000203180D1412001508AD
:10033000000203188D1412001508000203180D1591
:1003400012001508000203188D151200150800028E
:1003500003180D1612001508000203188D1612005E
:100360001508000203180D171200150800020318E3
:100370008D1708000310260DAF00C721B20008003A
:100380000310260D013EAF00C721B30008008130E5
:100390008A002F08D23E03188A0A820032088A0097
:1003A000330882008234123482341D34823425347E
:1003B00082342D348234353482343D3482344534B1
:1003C0008234513482345534823461348234653419
:1003D0008234713482347534823481348234853489
:1003E00082349134823495348234A1348234A534F9
:1003F0008234B1348234B5348234C1348234C53469
:100400008234D1348234D5348234E1348234E534D8
:100410008234F1348234F534833401348334053446
:10042000833411342D103030B10028181A2A0630C8
:10043000A600132B0130A600132B2818222A003007
:10044000A600132B0230A600132B28182A2A0030EE
:10045000A600132B0330A600132B2818322A0430D1
:10046000A600132B0330A600132B28183A2A0030BD
:10047000A600132B0530A600132B2818422A07309C
:10048000A600132B0030A600132B28184F2A00308B
:10049000310703194D2AB10B132B2D14132BA60171
:1004A000132B2808AC00A60A132B2C082806031DC2
:1004B0005B2AA601132B28182B10281C2B14A60A24
:1004C000132B2808AC00A60A132B2C082806031DA2
:1004D0006B2AA601132B28182A12281C2A16A60AF2
:1004E000132B2808AC00A60A132B2C082806031D82
:1004F0007B2AA601132B2818AA11281CAA15A60AC4
:10050000132B2808AC00A60A132B2C082806031D61
:100510008B2AA601132B28182A11281C2A15A60A93
:10052000132B2808AC00A60A132B2C082806031D41
:100530009B2AA601132B2818AA10281CAA14A60A65
:10054000132B2808AC00A60A132B2C082806031D21
:10055000AB2AA601132B28182A10281C2A14A60A35
:10056000132B2808AC00A60A132B2C082806031D01
:10057000BB2AA601132B2818A912281CA916A60A03
:10058000132B2808AC00A60A132B2C082806031DE1
:10059000CB2AA601132B28182912281C2916A60AD3
:1005A000132B2808AC00A60A132B2C082806031DC1
:1005B000DB2AA601132B2818A911281CA915A60AA5
:1005C000132B2808AC00A60A132B2C082806031DA1
:1005D000EB2AA601132B28182911281C2915A60A75
:1005E000132B2808AC00A60A132B2C082806031D81
:1005F000FB2AA601132B2818A910281CA914A60A47
:10060000132B2808AC00A60A132B2C082806031D60
:100610000B2BA601132B28182910281C2914A60A15
:10062000132BA60130140800AD100E1DAD140800E8
:10063000281090192814080027082602031C222BD2
:100640002608A70008002E10BD030310BC0CBB0C2D
:10065000BA0CB90C03182E140800B400B40B2E2BDE
:100660000800BA01BB01BC01A030B900B709371CB2
:100670003A143718BA14351E3A15351ABA15B51D7D
:100680003A16B519BA16351D3A173519BA17B51CE9
:100690003B14B518BB14351C3B153518BB15B61EDD
:1006A0003B16B61ABB16361E3B17361ABB17B61DBD
:1006B0003C14B619BC14361D3C153619BC15B61CB5
:1006C0003C16B618BC16361C3C173618BC17213021
:1006D000BD000800BE01BF010830C0000310C20CFD
:1006E000BF0DBE0DC10CBF0DBE0DC00B6E2B0800A3
:1006F000C3000000C30B792B0800CF0A4F08133C3E
:100700000319CF014F08B800FF01FE010800CF0315
:100710004F08013E031D8F2B1230CF00B800FF01A0
:10072000FE0108002908CF00B800ED3E031C9C2BF9
:100730001230CF024F08952BFF01FE010800C400C4
:100740002010201CA12BC40BA02B080051308400CA
:10075000003085002030C70000301A00C70BAD2BD9
:10076000C5014F0AC6000A304602031CBB2B0A30E3
:10077000C602C50AB32B1030C607C507731CC62BAB
:1007800051308400003085002430D4235730840059
:10079000003085004508D42312004608D423FF30DA
:1007A000E725FF30E7250800BE000708CA00060855
:1007B000CB004D30C8009730C9003E0803103E0DF5
:1007C000C8070318C90A0310BE0DBE0D0318C90AD5
:1007D0003E08C8070318C90A490887004808860068
:1007E0001600C10016001A00C10BF22B4A08870040
:1007F0004B088600080087308700013086004F0ACA
:10080000CE001600CC001600CD00CE0B012C4D08FA
:1008100086004C08CC1787000800F0304C02031DFE
:10082000182C4D087F072D24FF0F192CFE0A192CB8
:1008300016000800230095181B2C8B131515230098
:100840007F0891007D089300230055309600AA3060
:10085000960095148B17200008008B132300951821
:100860002F2C15112300910023009513151423003C
:10087000130820008B17080000302D24F300080017
:100880003C24731C452C7310462C73140030FF005D
:100890007308FD001A24A623A6230800FB23FF01EA
:1008A000FE010D24D000D0130D24F200F20A0D2415
:1008B000F400301C772C07302A02031D622C92238F
:1008C000B0014E2CAA08031D772C203029020319F1
:1008D0007D232130290203198723003029020319BF
:1008E000CF010C30290203194024B0014E2C2D08F1
:1008F00003198D2CA623A62303302D0203194024AF
:100900002D18852CAD18892C4E2C7D23A623A623CB
:100910007C2C8723A623A6237C2C0C3050020319A1
:10092000C6241630500284310319D724843118307C
:10093000500284310319F624843119305002853174
:1009400003190C2584311A30500285310319622DA8
:1009500084313D08003E031DB92CA01CB92CA01009
:10096000731CB42C7D234E2C0730B5003808B6001C
:100970003123F40B592C4E2C750D750D751A013A57
:10098000F51A013AF519013AF500080051308400D2
:10099000003085002030BE00BC24BC24BC24BC2414
:1009A000BC241A00BE0BCC2C7208E725080051307D
:1009B0008400003085002030F6000D241A00F60B6C
:1009C000DD2C7208E7257208E7257208E725720812
:1009D000E725080051308400003085001F30F60004
:1009E000120013001A00F60BF02C0800EA24603005
:1009F0008400003085000D248000703084000030B9
:100A000085000D2480007208E7257208E72572082A
:100A1000E7257208E72508000D24BE000708CA0074
:100A20000608CB00BE0820303E0203181A2D3E08EF
:100A3000BF005D2D2030BE024D30C8009730C90088
:100A40003E0803103E0DC8070318C90A0310BE0D67
:100A5000BE0D0318C90A3E08C8070318C90A490889
:100A60008700480886001600C1001600C000EA246E
:100A70004008F0004008E0003F1CF0013F1DE0018D
:100A8000BF18F009BF19E0097208E7257208E725C9
:100A90007208E7257208E725C10B352DEA24F0011D
:100AA000E001BF18F009BF19E0097208E7257208D4
:100AB000E7257208E7257208E7254A0887004B08F2
:100AC0008600080051308400003085002030BF00CF
:100AD0000D241A00BF0B682D6430BF00F030840075
:100AE000203085005108B5255208B5255308B52595
:100AF0005408B5255508B5255608B5255708B52518
:100B00005808B5255908B5255A08B5255B08B525F7
:100B10005C08B5255D08B5255E08B5255F08B525D7
:100B20006008B5256108B5256208B5256308B525B7
:100B30006408B5256508B5256608B5256708B52597
:100B40006808B5256908B5256A08B5256B08B52577
:100B50006C08B5256D08B5256E08B5256F08B52557
:100B60007008B525BF0B6E2DA92CBE00BE1BDF255E
:100B7000BE1FE32512003E1BDF253E1FE3251200AA
:100B8000BE1ADF25BE1EE32512003E1ADF253E1EDB
:100B9000E3251200BE19DF25BE1DE32512003E1914
:100BA000DF253E1DE3251200BE18DF25BE1CE32510
:100BB00012003E18DF253E1CE32512000800800AC3
:100BC0000319800908008008031D80030800F10054
:100BD000F03084002030850051082F2652082F263F
:100BE00053082F2654082F2655082F2656082F263F
:100BF00057082F2658082F2659082F265A082F261F
:100C00005B082F265C082F265D082F265E082F26FE
:100C10005F082F2660082F2661082F2662082F26DE
:100C200063082F2664082F2665082F2666082F26BE
:100C300067082F2668082F2669082F266A082F269E
:100C40006B082F266C082F266D082F266E082F267E
:100C50006F082F2670082F2671089F230800F600C2
:100C60000030F61BFF301A000030761BFF301A00F0
:100C70000030F61AFF301A000030761AFF301A00E2
:100C80000030F619FF301A0000307619FF301A00D4
:100C90000030F618FF301A0000307618FF301A00C6
:100CA00008000030D1000030D2008030D300FF3087
:100CB000E7250030D300FF30E7258030D300FF3038
:100CC000E7250030D300FF30E7258030D300FF3028
:100CD000E72502302602031C0301D1000030D200B8
:100CE0000130E7252D080319872EA701A6013D082D
:100CF000003E031D722E2D08D200D1012D08D40014
:100D00000130E725B5010C30B6003123722E301CBE
:100D1000692EB001F030D100D2017F30E725D1013A
:100D2000D2013F30E725F030D100D2017F30E725F6
:100D30002908D1002A08D200FF30E725FF30E72537
:100D4000A701A601692E8C019501CF01BD01AB0160
:100D5000AA01A901AC01A601A701B001A1010430BB
:100D6000A100A201A301AD017230210099008230DF
:100D70002100950023008C0122008C0121008C01B0
:100D800022008D0123008D0121008D0122008E01A2
:100D900021001C308E0022009001210001309000C3
:100DA0002000AD011D30F5008B168B1751308400EB
:100DB0000030850020002030F600FF301A00F60BCE
:100DC000DE2EFF30E725FF30E7255130840000306C
:100DD00085002030F60000301A00F60BEC2EFF30B4
:100DE000E725FF30E725FF30E7253C242D08D2001A
:100DF000FF30E725FF30E7254E2C2D1C4E2C4024DC
:100E0000512E8734273487343D3487344034873437
:100E10008A348734C1348734EB34883403348834DB
:100E20002734883468348E346B3490346E34903484
:100E3000B134913454349134D7349234DA34933415
:100E40005D34943460349634A334973406341934C2
:100E50000F3413340534203420344D347534733456
:100E6000653443346F346E3401342E346F3472344D
:100E7000673420342034203420340C347F34003460
:100E800019340F3447340134203420344D34753450
:100E90007334653463346F346E3420343334203427
:100EA0002D342034053420344E3475347434753484
:100EB000723469346E34673420344F34753472348C
:100EC00020344D3475347334653473342034203415
:100ED00041347534673475347334743420343234A7
:100EE0002D343434203432343034313433342034FB
:100EF000203420345334653461346E3461346E34BC
:100F000020344D3463344734753469347234653475
:100F10002034203419340F34343404342034203451
:100F200049342034773465346E3474342034743466
:100F30006F3420344D3475347334653463346F3416
:100F40006E34203461346E34643420346234753449
:100F500069346C34743420347434683469347334D0
:100F60002034053463346F346F346C3420340134EE
:100F700062346C3469346E346B34693465342034D3
:100F8000203419340F34273401342034203473349E
:100F90006F3420346D3461346E34793420346234EB
:100FA0006C3469346E346B346934653473342C3486
:100FB0002034043473346F3420346C346934743422
:100FC00074346C3465342034743469346D3465346D
:100FD0002E342034203419340F34153401342034A5
:100FE00020347734773477342E3404343234643414
:100FF0006B3469347434733401342E3463346F3495
:101000006D342034203419340F3421340134203429
:1010100020344D3475347334653443346F346E3456
:101020002034333420342D342034053441347534A5
:101030006734753473347434203432342D3434349A
:1010400020343234303431343334203420341834C2
:101050000F341F34013400340334003407340034B7
:101060000F3400341F3400343F3400347F340034F4
:10107000FF3400347F3480343F34C0341F34E034D4
:101080000F34F0340734F8340334FC340134FE34C4
:101090000034FF340134FF340334FF340734FF34A9
:1010A0000F34FF341F34FF343F34FF347F34FF34B8
:1010B000FF34FF347F347F343F343F341F341F34D8
:1010C0000F340F340734073403340334013401344C
:1010D00016341F343034FF3400340034003400340C
:1010E0000034003400340034003400340034003460
:1010F0000034003400340034003400340034003450
:10110000003400340034003400340034003400343F
:101110000034003400340034FF3400340034003430
:10112000003400340034003400340034003400341F
:10113000003400340034003400340034003400340F
:1011400000340034003400340034003400340034FF
:1011500000340034003400340034FF3400340034F0
:1011600000340034003400340034003400340034DF
:1011700000340034003400340034003400340034CF
:1011800000340034003400340034003400340034BF
:10119000003400340034003400340034FF340034B0
:1011A000003400340034003400340034003400349F
:1011B000003400340034003400340034003400348F
:1011C000003400340034003400340034003400347F
:1011D0000034003400340034003400340034FF3470
:1011E000003400340034003400340034003400345F
:1011F000003400340034003400340034003400344F
:10120000003400340034003400340034003400343E
:10121000003400340034003400340034003400342E
:10122000FF3400340034003400340034003400341F
:10123000003400340034003400340034003400340E
:1012400000340034003400340034003400340034FE
:1012500000340034003400340034003400340034EE
:101260000034FF34003400340034003400340034DF
:1012700000340034003400340034003400340034CE
:1012800000340034003400340034003400340034BE
:1012900000340034003400340034003400340034AE
:1012A00000340034FF34003400340034003400349F
:1012B000003400340034003400340034003400348E
:1012C000003400340034003400340034003400347E
:1012D000003400340034003400340034003400346E
:1012E000003400340034FF3400340034003400345F
:1012F000003400340034003400340034003400344E
:10130000003400340034003400340034003400343D
:10131000003400340034003400340034003400342D
:101320000034003400340034FF340034003400341E
:10133000003400340034003400340034003400340D
:1013400000340034003400340034003400340034FD
:1013500000340034003400340034003400340034ED
:1013600000340034003400340034FF3400340034DE
:1013700000340034003400340034003400340034CD
:1013800000340034003400340034003400340034BD
:1013900000340034003400340034003400340034AD
:1013A000003400340034003400340034FF3400349E
:1013B000003400340034003400340034003400348D
:1013C000003400340034003400340034003400347D
:1013D000003400340034003400340034003400346D
:1013E0000034003400340034003400340034FF345E
:1013F000003400340034003400340034003400344D
:10140000003400340034003400340034003400343C
:10141000003400340034003400340034003400342C
:10142000003400340034003400340034003400341C
:10143000FF3400340034003400340034003400340D
:1014400000340034003400340034003400340034FC
:1014500000340034003400340034003400340034EC
:1014600000340034003400340034003400340034DC
:101470000034FF34003400340034003400340034CD
:1014800000340034003400340034003400340034BC
:1014900000340034003400340034003400340034AC
:1014A000003400340034003400340034003400349C
:1014B00000340034FF34003400340034003400348D
:1014C000003400340034003400340034003400347C
:1014D000003400340034003400340034003400346C
:1014E000003400340034003400340034003400345C
:1014F000003400340034FF3400340034003400344D
:10150000003400340034003400340034003400343B
:10151000003400340034003400340034003400342B
:10152000003400340034003400340034003400341B
:101530000034003400340034FF340034003400340C
:1015400000340034003400340034003400340034FB
:1015500000340034003400340034003400340034EB
:1015600000340034003400340034003400340034DB
:1015700000340034003400340034FF3400340034CC
:1015800000340034003400340034003400340034BB
:1015900000340034003400340034003400340034AB
:1015A000003400340034003400340034003400349B
:1015B000003400340034003400340034FF3400348C
:1015C000003400340034003400340034003400347B
:1015D000003400340034003400340034003400346B
:1015E000003400340034003400340034003400345B
:1015F0000034003400340034003400340034FF344C
:10160000003400340034003400340034003400343A
:10161000003400340034003400340034003400342A
:10162000003400340034003400340034003400341A
:10163000003400340034003400340034003400340A
:10164000FF340034003400340034003400340034FB
:1016500000340034003400340034003400340034EA
:1016600000340034003400340034003400340034DA
:1016700000340034003400340034003400340034CA
:101680000034FF34003400340034003400340034BB
:1016900000340034003400340034003400340034AA
:1016A000003400340034003400340034003400349A
:1016B000003400340034003400340034003400348A
:1016C00000340034FF34003400340034003400347B
:1016D000003400340034003400340034003400346A
:1016E000003400340034003400340034003400345A
:1016F000003400340034003400340034003400344A
:10170000003400340034FF3400340034003400343A
:101710000034003400340034003400340034003429
:101720000034003400340034003400340034003419
:101730000034003400340034003400340034003409
:101740000034003400340034FF34003400340034FA
:1017500000340034003400340034003400340034E9
:1017600000340034003400340034003400340034D9
:1017700000340034003400340034003400340034C9
:1017800000340034003400340034FF3400340034BA
:1017900000340034003400340034003400340034A9
:1017A0000034003400340034003400340034003499
:1017B0000034003400340034003400340034003489
:1017C000003400340034003400340034FF3400347A
:1017D0000034003400340034003400340034003469
:1017E0000034003400340034003400340034003459
:1017F0000034003400340034003400340034003449
:101800000034003400340034003400340034FF3439
:101810000034003400340034003400340034003428
:101820000034003400340034003400340034003418
:101830000034003400340034003400340034003408
:1018400000340034003400340034003400340034F8
:10185000FF340034003400340034003400340034E9
:1018600000340034003400340034003400340034D8
:1018700000340034003400340034003400340034C8
:1018800000340034003400340034003400340034B8
:101890000034FF34003400340034003400340034A9
:1018A0000034003400340034003400340034003498
:1018B0000034003400340034003400340034003488
:1018C0000034003400340034003400340034003478
:1018D00000340034FF340134013401340134013464
:1018E0000134013401340134013401340134013450
:1018F0000134013401340034003400340034003445
:101900000034003400340034003400340034003437
:10191000003400340034023402340234023402341D
:101920000234023402340234023402340234023407
:101930000234023402340034003400340034003401
:1019400000340034003400340034003400340034F7
:1019500000340034003404340434043404340434D3
:1019600004340434043404340434043404340434B7
:1019700004340434043400340034003400340034BB
:1019800000340034003400340034003400340034B7
:10199000003400340034083408340834083408347F
:1019A0000834083408340834083408340834083457
:1019B000083408340834003400340034003400346F
:1019C0000034003400340034003400340034003477
:1019D0000034003400341034103410341034103417
:1019E00010341034103410341034103410341034D7
:1019F0001034103410340034003400340034003417
:101A00000034003400340034003400340034003436
:101A10000034003400342034203420342034203486
:101A20002034203420342034203420342034203416
:101A300020342034203400340034003400340034A6
:101A400000340034003400340034003400340034F6
:101A500000340034003440344034403440344034A6
:101A600040344034403440344034403440344034D6
:101A70004034403440340034003400340034003406
:101A800000340034003400340034003400340034B6
:101A90000034003400348034803480348034803426
:101AA0008034803480348034803480348034803496
:101AB0008034803480340034003400340034003406
:101AC0000034003400340034003400340034003476
:101AD0000034003400340034003400340034003466
:101AE0000034003400340034003400340034003456
:101AF0000034003400340134013401340134013441
:101B0000013401340134013401340134013401342D
:101B10000134013401340034003400340034003422
:101B20000034003400340034003400340034003415
:101B300000340034003402340234023402340234FB
:101B400002340234023402340234023402340234E5
:101B500002340234023400340034003400340034DF
:101B600000340034003400340034003400340034D5
:101B700000340034003404340434043404340434B1
:101B80000434043404340434043404340434043495
:101B90000434043404340034003400340034003499
:101BA0000034003400340034003400340034003495
:101BB000003400340034083408340834083408345D
:101BC0000834083408340834083408340834083435
:101BD000083408340834003400340034003400344D
:101BE0000034003400340034003400340034003455
:101BF00000340034003410341034103410341034F5
:101C000010341034103410341034103410341034B4
:101C100010341034103400340034003400340034F4
:101C20000034003400340034003400340034003414
:101C30000034003400342034203420342034203464
:101C400020342034203420342034203420342034F4
:101C50002034203420340034003400340034003484
:101C600000340034003400340034003400340034D4
:101C70000034003400344034403440344034403484
:101C800040344034403440344034403440344034B4
:101C900040344034403400340034003400340034E4
:101CA0000034003400340034003400340034003494
:101CB0000034003400348034803480348034803404
:101CC0008034803480348034803480348034803474
:101CD0008034803480341A3402341034FF340034B9
:101CE0000034003400340034003400340034003454
:101CF000003400340034FF34FF34FF340034003447
:101D0000003400340034FF34FF34FF34FF34003437
:101D1000003400340034003400340034FF34FF3425
:101D20000034003400340034003400340034003413
:101D30000034003400340034FF34FF340034003405
:101D40000034003400340034FF34FF34FF34FF34F7
:101D5000003400340034003400340034FF34FF34E5
:101D6000FF340034003400340034003400340034D4
:101D700000340034003400340034FF3400340034C4
:101D800000340034003400340034FF34FF34FF34B6
:101D9000FF3400340034003400340034FF34FF34A6
:101DA000FF34FF3400340034003400340034003495
:101DB0000034003400340034003400340034003483
:101DC000003400340034003400340034FF34FF3475
:101DD000FF34FF3400340034003400340034FF3466
:101DE000FF34FF34FF340034003400340034003456
:101DF0000034003400340034003400340034003443
:101E00000034003400340034003400340034FF3433
:101E1000FF34FF34FF340034003400340034003425
:101E2000FF34FF34FF34FF34003400340034003416
:101E30000034003400340034003400340034003402
:101E400000340034003400340034003400340034F2
:101E5000FF34FF34FF34FF340034003400340034E6
:101E60000034FF34FF34FF34FF34003400340034D6
:101E700000340034003400340034003400340034C2
:101E800000340034003400340034003400340034B2
:101E90000034FF34FF34FF34FF34003400340034A6
:101EA00000340034FF34FF34FF34FF340034003496
:101EB0000034003400340034003400340034003482
:101EC0000034003400340034003400340034003472
:101ED00000340034FF34FF34FF34FF340034003466
:101EE000003400340034FF34FF34FF34FF34003456
:101EF000003400340034003400340034FF34003443
:101F00000034003400340034003400340034003431
:101F1000003400340034FF34FF34FF340034003424
:101F20000034003400340034FF34FF34FF34FF3415
:101F3000003400340034003400340034FF34FF3403
:101F400000340034003400340034003400340034F1
:101F50000034003400340034FF34FF3400340034E3
:101F600000340034003400340034FF34FF34FF34D4
:101F7000FF3400340034003400340034FF34FF34C4
:101F8000FF340034003400340034003400340034B2
:101F900000340034003400340034FF3400340034A2
:101FA000003400340034003400340034FF34FF3493
:101FB000FF34FF340034003400340034FF34FF3485
:101FC000FF34FF3400340034003400340034003473
:101FD0000034003400340034003400340034003461
:101FE0000034003400340034003400340034FF3452
:101FF000FF34FF34FF340034003400340034FF3445
:10200000FF34FF34FF340034003400340034003433
:102010000034003400340034003400340034003420
:102020000034003400340034003400340034003410
:10203000FF34FF34FF34FF34003400340034003404
:10204000FF34FF34FF34FF340034003400340034F4
:1020500000340034003400340034003400340034E0
:1020600000340034003400340034003400340034D0
:102070000034FF34FF34FF34FF34003400340034C4
:102080000034FF34FF34FF34FF34003400340034B4
:1020900000340034003400340034003400340034A0
:1020A0000034003400340034003400340034003490
:1020B00000340034FF34FF34FF34FF340034003484
:1020C00000340034FF34FF34FF34FF340034003474
:1020D000003400340034003400340034163440340A
:1020E0000234AA34AA34AA34AA34AA34AA34AA34A8
:1020F000AA34AA34AA34AA34AA34AA34AA34AA34F0
:10210000AA34553455345534553455345534553432
:102110005534553455345534553455345534553477
:102120005534553455345534553455345534553467
:102130005534553455345534553455345534553457
:102140005534AA34AA34AA34AA34AA34AA34AA34F4
:10215000AA34AA34AA34AA34AA34AA34AA34AA348F
:10216000AA341634403405340034003400340034CA
:1021700000340034003400340034003400340034BF
:1021800000340034003400340034003400340034AF
:10219000003418343C341E343C34183400340034D9
:1021A000003400340034003400340034003400348F
:1021B000003400340034003400340034003400347F
:1021C000003400340034003400340034003400346F
:1021D00038347C347E343F343F347E347C3438347D
:1021E000003400340034003400340034003400344F
:1021F000003400340034003400340034003400343F
:102200000034003400340034003418343C341E34BC
:102210003C341834003400340034003400340034CA
:10222000003400340034003400340034003400340E
:1022300000340034003400340034003400340034FE
:10224000003400340034003438347C347E343F347D
:102250003F347E347C343834003418343C341E34FB
:102260003C3418340034003400340034003400347A
:1022700000340034003400340034003400340034BE
:1022800000340034003400340034003400340034AE
:10229000003400340034003438347C347E343F342D
:1022A0003F347E347C3438341634403404340034C3
:1022B000003400340034003400340034003400347E
:1022C0000034003400340034003400340034FF346F
:1022D0008134813481348134813481348134813456
:1022E000813481348134813481348134FF34003449
:1022F000003400340034003400340034003400343E
:10230000003400340034003400340034003400342D
:102310007E344234423442344234423442344234D1
:10232000423442344234423442347E340034003445
:1023300000340034003400340034003400340034FD
:1023400000340034003400340034003400340034ED
:1023500000343C34243424342434243424342434C9
:1023600024342434243424343C3400340034003401
:1023700000340034003400340034003400340034BD
:1023800000340034003400340034003400340034AD
:10239000003400341834183418341834183418340D
:1023A0001834183418341834003400340034163417
:1023B00040340834803480344034203410341034B5
:1023C000203440348034803440342034103410348D
:1023D00020344034083408340434023401340134E5
:1023E000023404340834083404340234013401342F
:1023F0000234043440348034803440342034103487
:10240000103420344034803480344034203410344C
:1024100010342034083404340234013401340234DA
:1024200004340834083404340234013401340234EE
:102430000434083420344034803480344034203430
:10244000103410342034403480348034403420340C
:1024500010341034043402340134013402340434AE
:1024600008340834043402340134013402340434AE
:1024700008340834103420344034803480344034FC
:1024800020341034103420344034803480344034CC
:10249000203410340234013401340234043408345A
:1024A000083404340234013401340234043408346E
:1024B00008340434103410342034403480348034F0
:1024C000403420341034103420344034803480348C
:1024D00040342034013401340234043408340834E4
:1024E000043402340134013402340434083408342E
:1024F0000434023420341034103420344034803416
:10250000803440342034103410342034403480344B
:102510008034403401340234043408340834043440
:1025200002340134013402340434083408340434ED
:102530000234013440342034103410342034403418
:10254000803480344034203410341034203440340B
:1025500080344034023404340834083404340234FF
:1025600001340134023404340834083404340234AD
:102570000134023480344034203410341034203498
:1025800040348034803440342034103410342034CB
:1025900040348034043408340834043402340134C0
:1025A000013402340434083408340434023401346D
:1025B000013402341634403404348034C034E034FE
:1025C000F0340F340734033401348034C034E03441
:1025D000F0340F3407340334013400340034003451
:1025E000003400340034003400340034003400344B
:1025F0000034003400340034003408340C340E3419
:102600000F34F034E034C034803408340C340E34E9
:102610000F34F034E034C0348034003400340034FB
:10262000003400340034003400340034003400340A
:10263000003400340034003400340F340E340C34D1
:102640000834103430347034F0340F340E340C3419
:102650000834103430347034F03400340034003432
:1026600000340034003400340034003400340034CA
:1026700000340034003400340034F034703430342A
:10268000103408340C340E340F34F03470343034D9
:10269000103408340C340E340F3400340034003459
:1026A000003400340034003400340034003400348A
:1026B000003400340034003400341634403408341C
:1026C000003400340034FF3400340034003400346B
:1026D0000034003400340034FF340034003400345B
:1026E0000034003400340034003400340034183432
:1026F0001834003400340034003400340034003422
:1027000000340034FF34003400340034003400342A
:1027100000340034003400340034FF34003400341A
:1027200000340034003400340034003418342434CD
:1027300024341834003400340034003400340034BD
:102740000034FF34003400340034003400340034EA
:10275000003400340034003400340034FF340034DA
:10276000003400340034003400343C344234423409
:10277000423442343C3400340034003400340034F9
:10278000FF340034003400340034003400340034AA
:102790000034003400340034003400340034FF349A
:1027A00000340034003400347E3481348134813488
:1027B0008134813481347E34003400340034003478
:1027C0000034003400340034003400340034183451
:1027D0001834003400340034003400340034003441
:1027E000003400340034FF3400340034003400344A
:1027F0000034003400340034FF340034003400343A
:1028000000340034003400340034003418342434EC
:1028100024341834003400340034003400340034DC
:1028200000340034FF340034003400340034003409
:1028300000340034003400340034FF3400340034F9
:10284000003400340034003400343C344234423428
:10285000423442343C340034003400340034003418
:102860000034FF34003400340034003400340034C9
:10287000003400340034003400340034FF340034B9
:1028800000340034003400347E34813481348134A7
:102890008134813481347E34003400340034003497
:1028A000FF34003400340034003400340034003489
:1028B0000034003400340034003400340034FF3479
:1028C000163440341234063406347E342034103446
:1028D0000034063406347E3420341034003400349E
:1028E0000034003400340034003400340034003448
:1028F0000034063406347E34203410340034063478
:1029000006347E3420340C34FC344034203400341B
:10291000033403343F3410340834003400340034BA
:102920000034003400340034003400340034003407
:10293000033403343F341034083400340C340C3482
:10294000FC34403420347E342034103400340634D7
:1029500006347E3420341034003400340034003423
:1029600000340034003400340034003400340634C1
:1029700006347E34203410340034063406347E3479
:102980002034103400344034203400340334033411
:102990003F34103408340034003400340034003440
:1029A000003400340334003400340034033403347E
:1029B0003F341034083400340C340C34FC344034CC
:1029C00020340034003410340034063406347E34AD
:1029D0002034103400340034003400340034003427
:1029E00000340634063400340034063406347E34B1
:1029F000203410340034063406347E34203410344D
:102A00000034003400340034033403343F341034D1
:102A1000083400340034003400340034003400340E
:102A2000033403343F340034033403343F3410346C
:102A3000083400340C340C34FC344034203400347A
:102A4000003400340034063406347E34203410342C
:102A500000340034003400340034003400340634D0
:102A600006347E342034063406347E342034103468
:102A70000034063406347E342034103400340034FC
:102A80000034003400340C34FC344034203400343E
:102A90000034003400340034003400340C340C347E
:102AA000FC34403420340C34FC34403420340034C2
:102AB000033403343F341034083400340034003419
:102AC0000034003400347E342034103400340034B8
:102AD00000340034003400340034063406347E34CC
:102AE0002034103400347E34203410340034063462
:102AF00006347E3420341034003400340034003482
:102B000000340034003440342034003400340034C5
:102B100000340034003400340C340C34FC344034C1
:102B2000203400340334403420340034033403347C
:102B30003F3410340834003400340034003400349E
:102B400000340034033410340034003400340034D2
:102B5000003400340034063406347E34203410341B
:102B600000340634063410340034063406347E341F
:102B70002034103400340034003400340034003485
:102B80000034063406340034003400340034003499
:102B9000003400340C340C34FC3440342034003421
:102BA000033403343F340034033403343F341034EB
:102BB000083400340034003400340034003400346D
:102BC000033403343F340034003400340034003420
:102BD0000034063406347E34203410340034063495
:102BE00006347E342034063406347E3420341034E7
:102BF000003400340034003400340034003406342F
:102C000006347E3420340034003400340034003480
:102C1000033403343F341034083400340C340C349F
:102C2000FC34403420340C34FC3440342034003440
:102C30000034003400340034003400340C340C34DC
:102C4000FC34403420340034003400340034063482
:102C500006347E34203410340034063406347E3496
:102C60002034103400347E342034103400340034E6
:102C700000340034003400340034063406347E342A
:102C8000203410340034003400340034033403346E
:102C90003F341034083400340C340C34FC344034E9
:102CA0002034003400344034203400340034003404
:102CB00000340034003400340C340C34FC34403420
:102CC00020340034033400340034063406347E34B7
:102CD000203410340034063406347E34203410346A
:102CE0000034003400341034003400340034003434
:102CF000003400340034063406347E34203410347A
:102D00000034063406340034033403343F341034C2
:102D1000083400340C340C34FC3440342034003497
:102D20000034003400340034003400340034003403
:102D3000003400340C340C34FC344034203400347F
:102D4000033403343F3416341F3403340134013464
:102D5000073407340F340F347F347F340F340F348B
:102D60001F341F340734073403340334013401346F
:102D7000043404340834083440344034083408340B
:102D80001034103404340434023402340F340F3459
:102D9000033403343F343F34FF34FF341F341F34D3
:102DA000073407340F340F343F343F3408340834C9
:102DB000023402342034203480348034103410340F
:102DC0000434043408340834203420340334033405
:102DD0000F340F341F341F34FF34FF340F340F34DB
:102DE000073407341F341F340F340F3402340234D5
:102DF00008340834103410348034803408340834F3
:102E000004340434103410340834083419340F34C2
:102E100044340134203420342034203441344334C9
:102E20004B342034203420342034203405342034F2
:102E3000203420342034413443344B342034203483
:102E400020342034203404342034203420342034FE
:102E5000413443344B342034203420342034203463
:102E600001342034203420342034203420342034E1
:102E7000203420342034203420344E3441344B3438
:102E800020342034203420342034203420342034A2
:102E900020342034203420342034013400340034F1
:102EA0000034003400340134F2340034003400348F
:102EB00000340334E0340034E034003400340534AA
:102EC0002834FE342834FE34283405342434543471
:102ED000FE34543448340534C434C83410342634F1
:102EE000463405346C349234AA3484340A340334BE
:102EF000383444348234003400340234A034C034D2
:102F00000034003400340334823444343834003420
:102F100000340534283410347C341034283405341B
:102F2000103410347C341034103402340534063438
:102F300000340034003405341034103410341034AC
:102F400010340234063406340034003400340534BE
:102F50000434083410342034403404347C34823453
:102F600082347C34003403344234FE34023400347E
:102F70000034043446348A349234623400340434E5
:102F80004434823492346C34003405341834283498
:102F90004834FE3408340434E434A234A2349C347B
:102FA000003404343C34523492340C34003404344D
:102FB00080348E349034E034003404346C349234F1
:102FC00092346C34003404346034923492347C345F
:102FD00000340234363436340034003400340234E1
:102FE000353436340034003400340434103428349A
:102FF00044348234003405342834283428342834C6
:1030000028340434823444342834103400340534F1
:10301000403480348A349034603405344C349234F3
:103020009E3482347C3405343E3448348834483409
:103030003E340534FE349234923492346C34053488
:103040007C3482348234823444340534FE34823415
:10305000823482347C340534FE3492349234923497
:1030600092340534FE3490349034903490340534E6
:103070007C348234923492345C340534FE3410341F
:1030800010341034FE3403348234FE34823400347D
:1030900000340434043402340234FC340034053483
:1030A000FE3410342834443482340534FE3402347F
:1030B0000234023402340534FE34403430344034B7
:1030C000FE340534FE34403420341034FE340534EC
:1030D0007C348234823482347C340534FE3490343F
:1030E00090349034603405347C3482348A348434AF
:1030F0007A340534FE349034983494346234053490
:1031000064349234923492344C34053480348034B4
:10311000FE34803480340534FC340234023402340A
:10312000FC340534F834043402340434F8340534FF
:10313000FC3402341C340234FC340534C6342834E4
:1031400010342834C6340534E03410340E341034CE
:10315000E034053486348A349234A234C2340334E1
:10316000FE34823482340034003405344034203458
:10317000103408340434033482348234FE3400348E
:103180000034053420344034803440342034053455
:10319000013401340134013401340234C034A03428
:1031A000003400340034043404342A342A341E3405
:1031B00000340434FE34223422341C340034043409
:1031C0001C34223422342234003404341C3422349B
:1031D0002234FE34003404341C342A342A341834A3
:1031E0000034043410347E349034403400340434D9
:1031F0001834253425343E3400340434FE3410347D
:1032000020341E34003403342234BE3402340034FB
:1032100000340434023401342134BE340034043424
:10322000FE34083414342234003403348234FE343F
:1032300002340034003405341E3420341834203471
:103240001E3404343E34103420341E34003404342C
:103250001C34223422341C34003404343F342434EB
:1032600024341834003404341834243424343F34DF
:10327000003404343E341034203420340034043418
:1032800010342A342A3404340034033420347E3495
:1032900020340034003404343C34023402343C34EE
:1032A00000340534383404340234043438340534FA
:1032B0003C3402340C3402343C34053422341434AB
:1032C00008341434223405343834053405343E349B
:1032D0000034043426342A343234003400340334C5
:1032E00010346C348234003400340134FF34003440
:1032F000003400340034033482346C34103400342D
:103300000034043400343E343E343E3480340434DB
:103310007734413463344134F73404341434223480
:0633200014342234943441
:020000040001F9
:02000E0084E983
:02001000FFDE11
:02E0000001001D
:00000001FF
